:020000020000FC
:100000000C9434000C94640D0C94640D0C94640DE9
:100010000C94640D0C94640D0C94640D0C94FB0B07
:100020000C94640D0C94640D0C94640D0C94640D8C
:100030000C94640D0C94640D0C94640D0C94640D7C
:100040000C94640D0C94640D0C94640D0C94640D6C
:100050000C94640D0C94640D0C94640D0C94640D5C
:100060000C94640D0C94640DA8950FEF0DBF08E07F
:100070000EBF0E94C20C0E94600278940E94180178
:100080000FEFC02E0E94DD000E947C010C943D0009
:100090000590002009F0089500E00093BD050C9440
:1000A000C007EAECFAE10E944800071671F40E94CA
:1000B0004800061659F40E944800051641F431968E
:1000C0000591F491E02F0995089531963196309677
:1000D0000C94530070EF60EF41E018810E94A10082
:1000E000013021F40E9495000C946A00512F0E9467
:1000F00095001D30A9F03D2C18811D3089F00E941B
:10010000A1003D1441F4762F652F512F0E949500D8
:100110004395433089F718810E94A1003D1409F0EE
:1001200008950E9495000C948B00DB1541F4CA15CC
:1001300031F404E00093BD050C94C00708952197A5
:1001400008951F9300271D3011F40C94C4001F75EF
:10015000103011F40C94AE001C3019F401E00C9432
:10016000C500103112F40C94C5001B3512F00C942C
:10017000C50010341AF003E00C94C5001A3112F4D3
:1001800022F402E00C94C50004E0D02E1F910895E3
:10019000CF3329F447E00E9406010C94E20048E0C6
:1001A0000E941F0140E20E941F01412F0E941F0177
:1001B000C3951DE018830C94E2004EE30E940601F3
:1001C000D5E0CFE30E942601183011F31F3701F369
:1001D0001A3011F40C94E20018831D3069F0C0301D
:1001E00029F447E00E9406010C94E200CA95412FD1
:1001F0000E941F010C94E20008950E9428028F9330
:10020000492F0E9406014F9101D008950090C0002F
:1002100005FE0C9406010E94E705B6FF0C9415013B
:100220000090C00007FEFCCFBF7B4093C60008953E
:100230004DE00E9406014AE00E94060108954D30FB
:1002400019F40E94180108950C9406018895000085
:100250000091C00007FF0C9426011091C60008957C
:100260000E9435010E94180108954591442321F10F
:10027000483F21F40E945D010C943501493F31F45F
:10028000159045910E9477010C9435014A3F21F465
:100290000E9418010C9435014B3F51F4EF93FF93EA
:1002A000E0E2F0E20E943501FF91EF910C943501FC
:1002B0000E9406010C9435010895EF93FF931124D9
:1002C00045914A3049F04C3039F04A3F29F0493FD6
:1002D00019F013940C9460011A944CE3141A1194BD
:1002E000169440E20E947701FF91EF9108950E94D9
:1002F00006011A94E1F70895D5E0CFE30FEFA02EA1
:1003000005E0B02E18810E94A100023011F40C9477
:1003100064060E941801A1600C948F01AE7F8DB716
:100320008F3C28F408E00093BD050C94C0070E94A0
:100330006A005D30F9F05B33E9F0032D023049F4D7
:100340007F706F705F700E9443020E94D0010C9416
:100350008F017F756F755F75413039F4032D033060
:1003600021F40E94BC010C948F010E9451005D3069
:1003700009F00895A160089551545A312AF005E01A
:100380000093BD050C94C007505CA0FF19F40E94B7
:10039000D0010895F5E0E52F50810E94D001089525
:1003A0000F93F4E0EC2D5083CA940C2D033F28F4F6
:1003B00006E00093BD050C94C0070F9108950F93BC
:1003C000C3940C2D00302AF007E00093BD050C9477
:1003D000C007F4E0EC2D50810F9108950E94DF01D9
:1003E00007E005175AF001E0503021F0000F5A9550
:1003F0000C94F401502F0E94D00108950AE000935C
:10040000BD050E94C007703049F0705D472F0E9403
:100410000601603019F440E30E940601603021F0CB
:10042000605D462F0E940601505D452F0E94060127
:10043000089577276627545618F073950C941B027D
:100440005C595A5018F063950C942102565F089538
:10045000982F9695969596959695905D9A3308F077
:10046000995F8F70805D8A3308F0895F089596FDEB
:10047000975F9F7086FD875F8F70990F990F990F17
:10048000990F892B08957330B2F4723032F06630D0
:1004900092F4653012F0563072F4662321F00AE0CF
:1004A000500F6A9581F7772309F4089504E688943C
:1004B000500F7A95C0F701E00093BD050C94C0077A
:1004C000E8E6FDE10E94300108950E941801F4E081
:1004D000E4EFC091B905D091BA05FD1711F4EC17FE
:1004E00031F040810E941F0131970C946D020E94EF
:1004F00018010E941801ECEEFFE10E9435015091B5
:10050000B9057091BA05505071400E94D001572F23
:100510000E9419020E940302EAEFFFE10E943501E6
:100520000E94DF010E9419020E9403020E9418012A
:100530000895AE7F0E948F010E94DF010E94190280
:100540000E9403020E94180108950E948E0144E255
:100550000E9406010E94DF01852F0E94FD000E947B
:1005600018010895AE7F0E948F010E94DF01052FC0
:100570000E94DF01F5E0E52F00830895A2FF0C94AF
:100580007003AE7F0E948F010E94DF01452E0E9402
:10059000DF01652F0E94DF01552EF5E0E52F608316
:1005A000A062A860AA7F0895F5E0E52D00810415FA
:1005B00019F003950083A06108950E948E010E94A6
:1005C000DF01052F0E94DF01501721F055270E94FF
:1005D000D00108955FEF0E94D00108950E948E011E
:1005E00050E000B605FE51E00E94D00108950E943F
:1005F0008E010EEF0C1949F00E94DF015F930E94FB
:10060000DF01F52FEF910C9409030E94DF01E52F24
:10061000FF2750810E94D00108950E948E010DEFA6
:100620000C1961F00E94DF015F930E94DF015F936C
:100630000E94DF01FF91EF910C9425030E94DF01DE
:10064000052F0E94DF01E02FFF27508308950E94AD
:100650008E010E94DF01052F0E94DF01509F1120B3
:10066000F09921F4502D0E94D00108950FE00093DD
:10067000BD050E94C0070E948E010E94DF01552324
:10068000F099B9F0052F0E94DF01652F771B59E023
:10069000661F5A9551F0771F701B20F4700F8894D5
:1006A0000C94480308940C944803562F0E94D001E0
:1006B000089501E10093BD050E94C0070E948E01CC
:1006C0000E94DF01052F0E94DF01500FF09918F002
:1006D0000E94D00108950FE00093BD050E94C0075D
:1006E0000E948E010E94DF01052F0E94DF01501B36
:1006F000F0991BF00E94D001089500E10093BD0520
:100700000E94C0070E948E010E94DF01052F0E94F7
:10071000DF0150230E94D00108950E948E010E94A3
:10072000DF0156950E94D00108950E948E010E941B
:10073000DF01550F0E94D00108950E948E010E9492
:10074000DF01052F0E94DF01502B0E94D001089588
:100750000E948E010E94DF01052F0E94DF015027B9
:100760000E94D00108950E948E010E94DF015095E1
:100770000E94D00108950E948E010E94DF015195D0
:100780000E94D001089551E00E94D00108950E9476
:100790008E010E94DF01052F0E94DF0150170C948B
:1007A000D9030E948E010E94DF01052F0E94DF0104
:1007B000051750E042F739F30E94D00108950E94D6
:1007C0008E010E94DF01552309F0A26008950DB744
:1007D0000E5F0DBF0895A46008950E948E010895D4
:1007E000B260089598810E94950088810E94370226
:1007F000582F0E94D0010E9495000E948E010895FA
:100800000E948E010E94DF01CF93DF93D0E5C9EFF4
:10081000CA950000E9F7DA950000C9F75A95B1F7D3
:10082000DF91CF91089555270E94D0010E948E013B
:100830000E94DF0101E005172AF0F09850FF0895AB
:10084000F09A08950CE00093BD050E94C0070E9435
:100850008E010E94DF01452FF4E0E4EF8091B9059D
:100860009091BA050C943F04F91711F48E1708F50E
:1008700000810D3019F031970C94340431975527CD
:1008800066277727F91711F48E1798F410810E94C4
:10089000A100023031F4762F652F512F31970C943F
:1008A00042047F706F705F700E9443024517E1F64B
:1008B000089509E00093BD050C94C0070E94270429
:1008C000DF2FCE2F08950E942704A06C0895B2FF59
:1008D0000C946C04B1600895B26008950E948E017A
:1008E0000E94DF01452F0E940601089588950000AF
:1008F0000091C00007FFFACF5091C600533009F4B1
:10090000B2600E94D00108950E948E010E94DF0112
:1009100008E040E3551F08F441E378DC0A95C9F785
:100920000E941801089504EB5091BE05579508F4F4
:1009300050275093BE050E94D0010895D4E0C4EF23
:100940000FEFC02EA1600E94E705A5FF0C94AB0439
:100950006C2E7D2EAF7DA4FF0C94B104D72DC62D37
:10096000AF7EA6FF0C94B904D093BC05C093BB0521
:10097000AF7BA7FF0C94C004DF2FCE2FB460AF77FE
:10098000B0FF0C94C804C091BB05D091BC05BA7FE0
:10099000B1FF0C94D2040E94E205C091B905D09138
:1009A000BA05BD7F0091BA05D01721F40091B905B1
:1009B0000C17A0F418810E94A100A1FF0C94E5047B
:1009C000043019F021970C94A004AD7F023019F483
:1009D00021970C94A0040E948F01B2CF0895F4E0F7
:1009E000E4EFF093BA05E093B9050FEFC02EAA2704
:1009F000BB27F1E0E0E000E00193F430E8F3E43FEE
:100A0000D9F7F5E0E0E400E00193F530E8F3EA35EA
:100A1000D9F70E941801E0E2FDE10E94300108953B
:100A2000ECE2FFE10E943501E6E5FFE10E943501BD
:100A300000E1202EF4E0E4EF8F2F0E94FD008E2FC6
:100A40000E94FD004AE30E94060140E20E94060166
:100A5000F13011F4E030D9F080810E94FD0040E2D5
:100A60000E94060131972A9481F40E9418018F2F69
:100A70000E94FD008E2F0E94FD004AE30E940601A5
:100A800040E20E94060100E1202E0C9428050E94FD
:100A900018010E941801E2E7FFE10E9435018091F0
:100AA000BA050E94FD008091B9050E94FD000E94D8
:100AB0001801ECE2FFE10E9435010E94180108953F
:100AC000ECE2FFE10E943501E6E4FFE10E9435011E
:100AD00000E1202EF3E0EFEF8F2F0E94FD008E2F1C
:100AE0000E94FD004AE30E94060140E20E940601C6
:100AF0000F93E03000E0F0070F91F1F0F2BDE1BD9F
:100B0000F89A80B50E94FD0040E20E9406013197EC
:100B10002A9481F40E9418018F2F0E94FD008E2FCD
:100B20000E94FD004AE30E94060140E20E94060185
:100B300000E1202E0C9478050E941801ECE2FFE100
:100B40000E9435010E9418010895ECE2FFE10E9425
:100B50003501E2E3FFE10E94350100E1202EE0E4EF
:100B6000F5E08F2F0E94FD008E2F0E94FD004AE3CA
:100B70000E94060140E20E940601EA35D1F081910F
:100B80000E94FD0040E20E9406012A9481F40E9426
:100B900018018F2F0E94FD008E2F0E94FD004AE356
:100BA0000E94060140E20E94060100E1202E0C9402
:100BB000BD050E941801ECE2FFE10E9435010E9490
:100BC00018010895E4EEFFE10E94350108950090B8
:100BD000C00007FE0C94F7050091C600033111F424
:100BE000B06408950091C600033009F4B26008951E
:100BF000DF93D2E0DA950000E9F7DF910895DF9303
:100C0000D4E1DA950000E9F7DF910895CF93DF93FF
:100C1000D0E5C3EFCA950000000000000000D1F746
:100C2000CFEFCA95000000000000D9F7CCEFCA95BD
:100C30000000000000000000D1F716F06894E9CF32
:100C4000DA95E89431F7DF91CF910895D5E0CFE3BD
:100C5000552788279927BF7D1881CA9583951D3010
:100C600051F00E94A100023041F0B0620130A1F3C6
:100C700093950C942C06092F0895B5FF53950C9469
:100C80002C0604E00093BD050C94C00702E000931D
:100C9000BD050C94C0070BE00093BD0571C17F70CA
:100CA0006F705F700E9443020895D5E0CFE3E0309B
:100CB00069F308810083319721970D30C1F7F093D4
:100CC000BA05E093B90508950E942606543018F736
:100CD0008091B9059091BA05943021F4843F11F4C4
:100CE0000C94D306D5E0CFE3552766277727CA159E
:100CF00042F218810E94A100023031F4762F652F54
:100D0000512F21970C9477060E944F06452EE091B3
:100D1000B905F091BA05B77FBF7E772766275527BB
:100D200055243196F43011F4E53F69F010810E94AA
:100D3000A100043041F0023081F75394562F672F01
:100D4000712F0C949106052D033031F05394562FDA
:100D5000672F70E00C94A306B4FD0C94B206B0614A
:100D60000C948D060E944F064516F1F118F4B860F8
:100D70007F2E6E2EF43029F4E53F19F4B3FF0C9466
:100D8000D306B3FF0C94C806541538F40C941E0710
:100D9000F43019F6E53F09F60895F43021F4E53F03
:100DA00011F40C941E070E942606003009F40895E1
:100DB000D5E0CFE3E091B905F091BA05F13021F427
:100DC000E03011F40C94EF060881008331972197ED
:100DD0000D30A1F7F093BA05E093B905089502E04C
:100DE0000093BD050C94C0073197EF01D13021F479
:100DF000C03011F40C944106088121970D30B1F7F1
:100E00000E2F0C1B8091B9059091BA05800F80932D
:100E1000B90518F493959093B905D13011F4C03009
:100E200031F008810083219731970C940D070E94BF
:100E30002606003011F00C94640608950E942606E0
:100E4000003071F10091BA05013029F40091B90523
:100E50000050081720F2E091B905F091BA05DF2F94
:100E6000CE2FC81BD040D093BA05C093B905F71553
:100E700021F4E61511F40C944307008108832196B0
:100E800031960C943707D5E0CFE3F72DE62D319757
:100E9000088100830D3021F0319721970C94480789
:100EA0000895D4E0CFEFE091B905F091BA05CE1BDB
:100EB000DF0BF3E0EFEFEC17FD072CF4EEE8FFE1BA
:100EC0000E9430010895EEEAFFE10E9430010FEF29
:100ED000C02E5091B9050E94D0015091BA050E94D0
:100EE000D001D4E0CFEFF3E0EFEF0881F9990C9453
:100EF0007607F2BDE1BD00BDFA9AF99AD13011F43E
:100F0000C03051F031970F93E03000E0F0070F91BF
:100F100019F021970C9475070895E0EDFFE10E9408
:100F200030010E94EF04D4E0CFEFEFEFF3E0F99946
:100F30000C949707F2BDE1BDF89A00B50883D13053
:100F400011F4C03021F0319721970C9497070DEFE1
:100F5000C02E0E94DF015093BA05F52F0E94DF01D9
:100F60005093B905E52F0F93EF3F04E0F0070F9181
:100F700031F4E0ECFFE10E9430010E94EF0408959B
:100F80000E9418010091BD05000FE4EBFFE0E00FA7
:100F90000591F491E02FEE1FFF1F0E9435010FEF26
:100FA0000DBF08E00EBF0FEFC02EA0E0B0E00E9422
:100FB000180163C814102510411050106E108410D1
:100FC0009B10BA10E4100E11281141115811711123
:100FD0008A119D11AA11B811C311D111E111F21199
:100FE000009164000F770093640055270E94D001A0
:100FF0000E948E010E94DF0101E00517A2F002E0CD
:1010000050FD00E20093B800459A449A00270093EF
:10101000B90000950093BB0004E00093BC0004E914
:101020000093BC0008950CE00093BD050E94C0072A
:101030000091BC0002FF0C9447080E948E010E94A0
:10104000DF015093BB0005E80093BC000091BC0099
:1010500007FFFCCF0091B900087F083111F0003480
:1010600041F45091B9005695569556950E94D0017D
:101070000895003239F0083429F002E10093BD05EB
:101080000E94C00704E10093BD050E94C00703E170
:101090000093BD050E94C0070091BC0002FF0C94A4
:1010A00077080E948E010E94DF015093BB0005E883
:1010B0000093BC000091BC0007FFFCCF0091B90079
:1010C000087F083241F45091B900569556955695CF
:1010D0000E94D0010895003329F002E10093BD057C
:1010E0000E94C00704E10093BD050E94C00703E110
:1010F0000093BD050E94C0070091BC0002FF0C9444
:10110000AA0851E00E94D0010E948E010E94DF01D6
:1011100001E0051722F104EC50FF04E80093BC0045
:101120000091BC0007FFFCCF0091B900087F00359B
:1011300029F45091BB000E94D0010895003529F098
:1011400002E10093BD050E94C00704E10093BD05C4
:101150000E94C00703E10093BD050E94C0070CE098
:101160000093BD050E94C0070091BC0002FF0C94D3
:10117000CB0804EA0093BC000091BC0007FFFCCF41
:101180000091B900087F083009F4089502E1009346
:10119000BD050E94C00703E10093BD050E94C00782
:1011A0000091BC0002FF0C94E10804E90093BC002C
:1011B0000FEF0093BB00089502E10093BD050E946C
:1011C000C00703E10093BD050E94C0070091BC0069
:1011D00002FF0C94FF080091BC0004FF0C94F3087C
:1011E00050E80C94FC080091BC0007FFFCCF509124
:1011F000B9005695569556950E94D001089503E181
:101200000093BD050E94C007009164000B7F00930E
:10121000640052E00E94D0010E948E010E94DF0112
:1012200003E005174AF0550F550F0E947A090CB5D7
:10123000037F052B0CBD08950DE00093BD050E94B2
:10124000C0070E948E010E94DF0101E0051752F0E5
:101250000CB500620CBD50FD0C9431090CB50F7D2E
:101260000CBD08950CE00093BD050E94C0070E94CC
:101270008E010E94DF0107E0051782F0052E5370F2
:101280000CB5087F052B0CBD0DB501600DBD02FC32
:101290000C944D090DB50E7F0DBD08950AE0009325
:1012A000BD050E94C0070E948E010E94DF012A989E
:1012B000000000005EBD0DB407FE0C945B095EB536
:1012C00008952A98000000005EBD0DB407FE0C943E
:1012D00065095EB50E94D001089551E00E94D001D9
:1012E0000E948E010E94DF012A9A50FD0C94790918
:1012F0002A98089504B10C6204B905B1046005B9D7
:1013000001E50CBD0DB50E7F0DBD089500E0009305
:101310007B0055270E94D0010E948E010E94DF01B0
:1013200000917C00052B00937C0006EC00937A0072
:1013300000917A0006FD0C94980906EC00937A005F
:1013400000917A0006FD0C94A009509179000E944A
:10135000D001089555270E94D0010E948E010E945D
:10136000DF0101E005175AF000917C000F73006265
:1013700050FD0C94BC09006C00937C0008950CE0B7
:101380000093BD050E94C0070E94480AEF5DFF4F11
:1013900050810E94D00108950E94480AEF93FF9364
:1013A0000E948E010E94DF01FF91EF91EF5DFF4FE0
:1013B000508308950E94480AEF93FF930E948E0184
:1013C0000E94EE010E94DF01FF91EF91EF5DFF4F60
:1013D0000C944D0A0E94480AEF93FF930E948E01DD
:1013E0000E94EE010E94DF01FF91EF91EF5DFF4F40
:1013F0000C94510A0E94480AEF93FF930E948E01B9
:101400000E94DF01FF91EF91EE5DFF4F5083089541
:101410000E94480AE05EFF4F50810E94D00108956B
:101420000E94480AEF93FF930E948E010E94EE01F2
:101430000E94DF01FF91EF91EE5DFF4F0C944D0A8A
:101440000E94480AEF93FF930E948E010E94EE01D2
:101450000E94DF01FF91EF91EE5DFF4F0C94510A66
:101460000E94480AEF93FF930E948E010E94EE01B2
:101470000E94DF01FF91EF91E05EFF4F00810523A5
:1014800050E000230FB601FC51E00E94D001089506
:1014900003E05154509FF00108950081052B008313
:1014A0000895509500810523008308950E948E01C0
:1014B00001E80093800009E0009381000027009379
:1014C0008200219A0E94DF01002700938900509337
:1014D000880008950E948E0103E80093800009E0CF
:1014E00000938100002700938200219A0E94DF016F
:1014F000052F0E94DF015093890000938800089512
:10150000002700938000089555270E94D0010E9473
:101510008E010E94DF0107E005178AF00091BF05E8
:10152000087F502B5093BF05002700936F0006BB28
:1015300000938200009380000093810008950AE0E8
:101540000093BD051DDD51E00E94D0010E948E0177
:101550000E94DF0101E005174AF00091BF050F77F7
:1015600050FF01C000680093BF0508950CE0009390
:10157000BD0506DDCF93DF936627552756BB6093E5
:10158000850050938400B09A0091BF05702F707849
:10159000C894771F771F76600770E1EDFAE0E00FDF
:1015A00009947AC006C005C004C02AC029C028C05A
:1015B0004FC0033008F005E0709381006093850010
:1015C00050938400D8E0C3EFCA95000000000000EB
:1015D0000000D1F7CFEFCA95000000000000D9F756
:1015E000CCEFCA950000000000000000D1F716F013
:1015F0006894E9CFDA95E89431F70A9519F74CC069
:101600000350033008F005E070938100609385007B
:1016100050938400D0E5C3EFCA950000000000009D
:101620000000D1F7CFEFCA95000000000000D9F705
:10163000CCEFCA950000000000000000D1F716F0C2
:101640006894E9CFDA95E89431F70A9519F724C040
:101650007093810060938500509384000AE0D0E588
:10166000C3EFCA950000000000000000D1F7CFEFE3
:10167000CA95000000000000D9F7CCEFCA95000021
:10168000000000000000D1F716F06894E9CFDA9569
:10169000E89431F70A9519F750918400609185001C
:1016A000002700938100B09908C0C9E5D5E06883A0
:1016B0000E94D001DF91CF910895DF91CF910EE08C
:1016C0000093BD055DDC0E948E010E94DF01152F95
:1016D00088940E947B0B08950E948E010E94DF0176
:1016E000152F08940E947B0B08950E94A50B512F83
:1016F0000E94D001089504B1077E04B905B10861C4
:1017000005B979E01C9B0C94820B2D9A259810F05A
:101710002D98259A2C98249A0E94C60B24982C9ACE
:101720000E94C60B1C990C948A0B20F02D9A2598C8
:101730000C949C0B2D98259A1C9B0C949C0B259823
:101740002D9A111F7A95F1F6089504B1077E04B918
:1017500005B1086105B979E01C990C94AC0B88942B
:101760001D9B0C94BB0B08942C98249A1D990C94E7
:10177000B60B0C94C00B2C98249A1D9B0C94BD0B9B
:1017800024982C9A111F7A9539F7089580E590E5F1
:101790009A95F1F78A95D9F70895CF93DF93552756
:1017A0000E94D0010E948E010E94DF010517F2F015
:1017B00050FD0C94E70B0E94AA0CC3ECD5E00993F2
:1017C000099308835C9A5498DF91CF910895C7E5F7
:1017D000D5E00E94270C00270093C605549A5C9818
:1017E0000E948A0CDF91CF91789408950CE00093C9
:1017F000BD050E94C0077F937FB77F936F935F9370
:10180000EF93FF93FDE7E091C6055091C30560910A
:10181000C4057091C505E50EF61EE71F5491E093CF
:10182000C60550FF0C941E0C00005C9AFF91EF91CE
:101830005F916F917F917FBF7F9118955C98FF9129
:10184000EF915F916F917F917FBF7F911895C7E571
:10185000D5E077276627552700EF102E0880012056
:101860000294002049F080E0581F90E0691F00E0DA
:10187000701F0A940C94310C0990129401200020DE
:1018800049F089E9581F99E9691F09E1701F0A9415
:101890000C943F0C0880129401200294002049F01F
:1018A0008CE5581F9FE8691F02E0701F0A940C9492
:1018B0004E0C099012940120002049F089E8581F2D
:1018C00091E4691F00E0701F0A940C945C0C08807E
:1018D000129401200294002049F08DE8581F96E0F0
:1018E000691F00E0701F0A940C946B0C088012941E
:1018F0000120002041F087EA581F90E0691F00E0B6
:10190000701F0A94B1F75093C3056093C405709398
:10191000C5050895009164000F7B009364000027C3
:1019200007BB0093B2000093B0000093B100009396
:10193000B3000093B4000FE40093B30002E00093FF
:10194000B00001E00093B1000091700002600093CC
:1019500070000895F894002707BB0093B00000932F
:10196000B1000093B2000093B4000093B300009163
:1019700070000D7F0093700000916400006400937C
:1019800064000895A89504B7007004BF009160003A
:1019900008610093600000700093600006E204B9E3
:1019A00000E005B900E007B900E008B902E20AB9B1
:1019B00000E00BB900270093BF050EBBF09A54EB73
:1019C0000091000105270093BE0500E00093C500CB
:1019D00009E10093C40008E90093C10001E003BFDE
:1019E000439A0E94FF0533990EC043980E948D07C9
:1019F0000E949E040E9418010E941801E0E2FDE18D
:101A00000E94300108950E94EF040895E3E0F0E0A1
:101A100009E007BF049106950370003019F4E0E077
:101A2000F8E314C0013019F4E0E0FCE30FC0023029
:101A300019F4E0E0FEE30AC0033019F4E0E0FFE34C
:101A400005C00BE00093BD050C94C007EF93FF9316
:101A500008E0102EEE1FFF1F05910F3F19F0003018
:101A600009F007C01A94C1F705E10093BD050C9475
:101A7000C007E4E0F0E20E943501FF91EF918F2F63
:101A80000E94FD008E2F0E94FD000E9418010E94FE
:101A900018011124F8941DBA109268001CBC10BEE5
:101AA0001FBA10926E0010926F0010927000109288
:101AB000C1001092BC0010927A0014B817B81AB87E
:101AC00015B818B81BB8099418954C4953206502ED
:101AD00052554E209E045052494E99025052582061
:101AE000A502505242208404464F5220EB034E453B
:101AF0005854D40253495A2079024E455720EF04D6
:101B000050500B205E0350500D20700350500A209F
:101B1000270350500F203B03414F56201304454DDF
:101B200049546E04501A1D20B20250501D20BE02AE
:101B3000501C1E20DD0250501E20D10350501C208E
:101B4000C70350494620DF0350544F20ED03505047
:101B50000420F203454E4420F003414E442082030A
:101B60004C5352208D034C534C209503504F522020
:101B70009D03584F5220A803434F4D20B3034E45B9
:101B80004720BB03524E4420930444454C4100047B
:101B9000474F544F5E04474F5355630452455455C5
:101BA00067045448454EE7034B45592076044143AA
:101BB0004F20EE025341564551074C4F41448D078B
:101BC0005045454BF702504F4B450D034F444220C3
:101BD000CC0949444220C40953444220DA09434411
:101BE0004220EA094F504220FA0953424220100A8B
:101BF00043424220200A494E4220080A49424220DC
:101C0000300A4F444320CC0949444320C40953447B
:101C10004320DA0943444320EA094F504320FA099C
:101C200053424320100A43424320200A494E432096
:101C3000080A49424320300A4F444420CC09494411
:101C40004420C40953444420DA0943444420EA09A7
:101C50004F504420FA0953424420100A4342442082
:101C6000200A494E4420080A49424420300A44557B
:101C70004D5010054544554D60055644554DA5053C
:101C800044535245750B4453434F6C0B44534445E6
:101C9000630B49434720840A49434520A30A49432B
:101CA0005020BA0A50574D38560A505745206A0AF4
:101CB00050574F20800A44445320CD0B424C44528D
:101CC000060D41444320860941445220AA0953503D
:101CD0004D20040953504F20210953504320370908
:101CE00053505720530953505220610953505320E9
:101CF0006D0954574920F00754575320B4085457DE
:101D00005020D008545741201808545757204C08E9
:101D1000545752207C0854574220E6080000000027
:101D2000F93C3DFAF84174746F42415349432066CF
:101D30006F722041546D65676133323820FAF8566E
:101D400065723A20322E3131204275696C6420630D
:101D50006F64653A2032303132303330382E3033D0
:101D60003132FAF93C2D0000F84F726967696E61F3
:101D70006C20636F64652028432932303032206242
:101D80007920526963686172642043617070656C88
:101D900073FAF8687474703A2F2F70726F6A656303
:101DA00074732E63617070656C732E6F7267202080
:101DB00070726F6A656374734063617070656C7391
:101DC0002E6F726720FAF93C2DFAF8546865206688
:101DD0006F6C6C6F77696E672061726520656E68E5
:101DE000616E63656D656E74732062792053636FF5
:101DF000747420566974616C65FAF86B73765F7061
:101E0000726A40676D782E636F6D20FAF84D6567D2
:101E10006138382F3136382F3332382F333255343A
:101E200020706F727420284329323031312C3230C7
:101E3000313220FAF85457492F5350492F44445314
:101E4000202620496E707574204361707475726528
:101E5000202843293230313120FAF84D656761334B
:101E60003255342055534220262044465520426F97
:101E70006F746C6F6164657220737570706F7274CB
:101E8000202843293230313220FAF93C2DFAF84D1E
:101E90006567613136382F33323820426F6F746C8A
:101EA0006F61646572206261736564206F6E207378
:101EB000746B353030626F6F742E63FAF8436F7055
:101EC00079726967687420286329323030332C2096
:101ED0004A61736F6E20502E204B796C65FAF93C85
:101EE0002DFAF8416C6C2072696768747320616E1A
:101EF000642072656D6564696573206578707265CC
:101F000073736C79207265736572766564FAF84E46
:101F10006F7420666F7220636F6D6D6572636961A7
:101F20006C20757365FAF93C3DFA0000F9352DFA1D
:101F300000005661726961626C657320696E20529F
:101F4000414D3AFA000045455020436F6E74656E6E
:101F500074733AFA000050524F4752414D204D657C
:101F60006D6F727920436F6E74656E74733AFA0008
:101F700000004E65787420617661696C61626C6501
:101F8000206C6F636174696F6E3A20000000FB3A49
:101F90002050726F6772616D20746F6F206C617278
:101FA000676520666F722045455021FA0000536135
:101FB00076696E6720746F204545502EFA00000048
:101FC000FB4545502065726173656421FA0000008D
:101FD0004C6F6164696E672066726F6D2045455075
:101FE000FA000000427265616BFA00004672656596
:101FF0003A2070616765733A00002063686172730C
:102000003A000000FA496E766F6B696E6720626F66
:102010006F746C6F616465722061742030780000A9
:102020004572726F72200000FB303A20556E6B6E65
:102030006F776E20636F6D6D616E64206F72206FBD
:1020400070657261746F722E0000FB313A20456E2C
:10205000636F756E746572656420612076616C755E
:10206000652074686174206973206E6F74206265E6
:10207000747765656E203020616E64203235352EB0
:102080000000FB323A2050726F6772616D206D65FF
:102090006D6F72792069732066756C6C2E0000007C
:1020A000FB333A20456E636F756E7465726564200C
:1020B0006120636861726163746572207468617421
:1020C000206973206E6F742061207265636F676E84
:1020D000697A656420747970652E0000FB343A6972
:1020E0006E7465726E616C206572726F72202D2045
:1020F000627566666572206C696D697420657863C7
:102100006565646564000000FB353A20496E6170C6
:1021100070726F7072696174652076617269616254
:102120006C65206E616D6520656E636F756E74659C
:102130007265642E0000FB363A204461746120739E
:102140007461636B2070757368206572726F7220A2
:102150002D20746F6F206D616E7920617267756DCF
:10216000656E7473206F6E206F6E65206C696E658E
:102170002E000000FB373A204461746120737461C3
:10218000636B20706F70206572726F722EFAF9099E
:102190002046756E6374696F6E2074726965642081
:1021A000746F2075736520612076616C756520748D
:1021B00068617420776173206E6F74206176616945
:1021C0006C61626C652E0000FB383A204D616368DB
:1021D000696E6520737461636B206572726F72FA49
:1021E000F9092046756E6374696F6E7320616E64C1
:1021F0002F6F722063616C6C73206E6573746564FD
:1022000020746F6F20646565706C79206F72207424
:102210006F6F20636F6D706C65780000FB393A203A
:10222000474F544F206F7220474F535542206465EB
:102230007374696E6174696F6E206C696E65207766
:102240006173206E6F7420666F756E642E000000DF
:10225000FB413A2053706563696669656420626971
:102260007420706F736974696F6E2072616E676538
:10227000206F6620303A3720657863656564656451
:102280000000FB423A204C696E65206E756D6265F8
:102290007220686173206D6F7265207468616E20B2
:1022A0007468726565206E756D6572616C7300008F
:1022B000FB433A205370656369666965642062690F
:1022C0007420706F736974696F6E2072616E6765D8
:1022D000206F6620303A31206578636565646564F7
:1022E0000000FB443A2053706563696669656420A9
:1022F00062697420706F736974696F6E2072616EA9
:102300006765206F6620303A3320657863656564C1
:1023100065640000FB453A20496E70757420436186
:102320007074757265207265676973746572206F69
:10233000766572666C6F77000000FB463A2041724A
:102340006974686D65746963206F766572666C6F19
:1023500077000000FB31303A2041726974686D6586
:1023600074696320756E646572666C6F7700000037
:10237000FB31313A20446976696465206279207ABC
:1023800065726F000000FB31323A205457492062D9
:102390007573206572726F72206F63637572656406
:1023A0000000FB31333A2054574920696E7465723E
:1023B00066616365206E6F7420656E61626C656432
:1023C0000000FB31343A2054574920536C61766544
:1023D000207265706C6965642077697468204E416D
:1023E0004B000000FB31353A204E6F20426F6F7476
:1023F0002D6C6F6164657220666F756E64000000FD
:107D00000000000000000000000000000000000073
:107D10000000000000000000000000000000000063
:107D20000000000000000000000000000000000053
:107D30000000000000000000000000000000000043
:107D40000000000000000000000000000000000033
:107D50000000000000000000000000000000000023
:107D60000000000000000000000000000000000013
:107D70000000000000000000000000000000000003
:107D8000FFFFFFFFFFFFFFFFFFFFFFFFFFFFFFFF03
:107D9000FFFFFFFFFFFFFFFFFFFFFFFFFFFFFFFFF3
:107DA000FFFFFFFFFFFFFFFFFFFFFFFFFFFFFFFFE3
:107DB000FFFFFFFFFFFFFFFFFFFFFFFFFFFFFFFFD3
:107DC000FFFFFFFFFFFFFFFFFFFFFFFFFFFFFFFFC3
:107DD000FFFFFFFFFFFFFFFFFFFFFFFFFFFFFFFFB3
:107DE000FFFFFFFFFFFFFFFFFFFFFFFFFFFFFFFFA3
:107DF000FFFFFFFFFFFFFFFFFFFFFFFFFFFFFFFF93
:107E0000112484B714BE81FFF0D085E080938100F7
:107E100082E08093C00088E18093C10086E0809377
:107E2000C20080E18093C4008EE0C9D0259A86E02C
:107E300028E13EEF91E0309385002093840096BBCB
:107E4000B09BFECF1D9AA8958150A9F7CC24DD24C4
:107E500088248394B5E0AB2EA1E19A2EF3E0BF2EE7
:107E6000A2D0813461F49FD0082FAFD0023811F036
:107E7000013811F484E001C083E08DD089C08234E0
:107E800011F484E103C0853419F485E0A6D080C0E4
:107E9000853579F488D0E82EFF2485D0082F10E0AE
:107EA000102F00270E291F29000F111F8ED06801E7
:107EB0006FC0863521F484E090D080E0DECF843638
:107EC00009F040C070D06FD0082F6DD080E0C81688
:107ED00080E7D80618F4F601B7BEE895C0E0D1E017
:107EE00062D089930C17E1F7F0E0CF16F0E7DF06D8
:107EF00018F0F601B7BEE89568D007B600FCFDCFD4
:107F0000A601A0E0B1E02C9130E011968C91119780
:107F100090E0982F8827822B932B1296FA010C0160
:107F200087BEE89511244E5F5F4FF1E0A038BF0790
:107F300051F7F601A7BEE89507B600FCFDCF97BE46
:107F4000E89526C08437B1F42ED02DD0F82E2BD052
:107F50003CD0F601EF2C8F010F5F1F4F84911BD097
:107F6000EA94F801C1F70894C11CD11CFA94CF0C13
:107F7000D11C0EC0853739F428D08EE10CD085E9AC
:107F80000AD08FE07ACF813511F488E018D01DD067
:107F900080E101D065CF982F8091C00085FFFCCF94
:107FA0009093C60008958091C00087FFFCCF809118
:107FB000C00084FD01C0A8958091C6000895E0E648
:107FC000F0E098E1908380830895EDDF803219F02E
:107FD00088E0F5DFFFCF84E1DECF1F93182FE3DFCA
:107FE0001150E9F7F2DF1F91089580E0E8DFEE27F6
:067FF000FF2709940404C0
:00000001FF
